:020000040000FA
:0A00000000000000A4EF00F0BAD0E9
:0800180007D10E6E960E056E75
:10002000980E066E6AD8D8B4CA90D8A4CA80FC0FBD
:10003000D8A0CA92D8B0CA82800E056E960E066EFF
:10004000980E096E0A6ACAB025D8CAB223D857D802
:100050000504CB6E05C007F006C008F000500B6E1B
:100060000C6E003C0C6A60D80A500E2E0AD0BE6E90
:100070000C0EBD6E09BEBD8A09BCBD889394CA84AE
:100080001200BB6E0C0EBA6E09BEBA8A09BCBA88E1
:100090009492F5D700D8D890093206320532120072
:1000A000E836E836FC0B0109C212C009C216C0507E
:1000B000F80B0309C06E320E15D8C282C2B2FED749
:1000C000C4CF12F0C350116E1200086A076EFF0E03
:1000D0000726082200D0D8A01200030E066EE60EF6
:1000E00002D8F5D7066AFE0F056EE86A065AD8A050
:1000F00012000000050600D0F8D70A6A096A100E3F
:10010000F36E063409360A360750095C08500A585F
:1001100005E30750095E08500A5AD88005360636AE
:10012000F32EEFD70550120007500B02F3CF09F062
:10013000F4CF0AF008500B02F3500A2607500C02C5
:10014000F3500A26095012004F0EAF6E240EAC6E0B
:10015000900EAB6E00010F0EC16E070EB46EC69A04
:10016000CF0E926EE00E936EC00E946E92849286C5
:10017000020EC06E0D0EC16E010EC26E6CD0F2A4E6
:1001800003D0F294817A11009EAA19D0060EAB1406
:1001900012E1E2CF60F0E1CF5FF0612A10EE80F073
:1001A0006150E126000EE222AECFE7FF60C0E2FF21
:1001B0005FC0E1FF1100AE50AE50AB98AB881100AC
:1001C0006150625C14E0622AEACF06F0E9CF05F0E4
:1001D00000EE80F06250E926000EEA22EF50056E34
:1001E00006C0EAFF05C0E9FFD880120004D0E86825
:1001F000056ED8A012001200616A626A9D8A9F8A09
:10020000F28EF28C12009D9A00EE80F0010EF46ED8
:10021000F36AF306000EF45AEE6AF450F310F9E1B3
:10022000616A626A9D8A1200F29EE0CF00F7D8CF21
:1002300001F7E8CF02F7F28E0001A192F29E00C70B
:10024000E0FF01C7D8FF02C7E8FFF28E10009EA8AA
:10025000FED7AD6E1200939A8A8A0A0E36DF929804
:100260008998929A899A94988B98949A8B9A949058
:100270008B9094968B96010EC26E000E11DF5B6E12
:1002800012C05CF0156A80B4152A156A80B6152A6A
:1002900093908A9093928A9293968A9693988A984A
:1002A0000068520E086E080E076E010EB6DE006A78
:1002B000520E086E080E076E020EAFDE366A356A01
:1002C000336A00EE68F0180EEE68E82EFDD7346A47
:1002D0004D6A7F0E4E6E4EC065F06690646A636A2A
:1002E0004A6A4B6A4C6A396A386A3B6A3A6A3D6ABA
:1002F0003C6A416A406A436A426A456A446A476A9C
:10030000466A496A486A366A77DF7DDFCD6AF294C9
:10031000F28A870ED56EB16AA192A082D08EA29287
:10032000B10EB16E56EC09F054EC0DF051EC0FF03B
:1003300046EC13F0030EC26E000EB2DE5B6E12C00E
:100340005CF0470E5C5C03E3BCEC08F003D022ECED
:1003500009F04D6A532AE86A53B2010F54B00108FC
:1003600006E154704F2A000E50225122522228DFFB
:10037000146EEA0E145C06E3FE0E145C01E2166ACB
:1003800030EF05F014AE38D0166A890E145C05E122
:1003900014C016F0176818682DD0990E145C05E18A
:1003A00014C016F019681A6825D0A90E145C05E16E
:1003B00014C016F01B681C681DD0B90E145C05E152
:1003C00014C016F01D681E6815D0C90E145C04E137
:1003D00014C016F01F680ED0D90E145C04E114C0CE
:1003E00016F0206807D0E90E145C04E114C016F082
:1003F000216822682FEF05F0165204E130EF05F076
:100400002FEF05F0890E165CD8A468D0172803E1F9
:1004100014C017F05FD014C018F0600E175C05E12F
:10042000339035908998369052D0610E175C05E173
:1004300033903590899A36804AD0620E175C08E175
:100440003390359036B002D0899801D0899A3FD048
:10045000630E175C07E13392339435923594369EE0
:100460008B9A35D0640E175C03E0650E175C08E1CB
:100470008B868B8036923694369A3686369827D07D
:10048000660E175C08E18B808B8636923694368632
:100490003698369A1CD0670E175C0AE13398359867
:1004A0008B983696369236948B908B9636980FD0E2
:1004B0007A0E175C0CE1006A520E086E080E076E89
:1004C000020E0DEC00F0339A359A496A486A1768B3
:1004D0002FEF05F030EF05F02FEF05F0990E165CC9
:1004E000D8A4FEEF04F0192804E114C019F0FCEFC1
:1004F00004F014C01AF01A52D8A462D0600E195C2D
:1005000005E1339035908998369056D0610E195C8C
:1005100005E133903590899A36804ED0620E195C91
:1005200008E13390359036B002D0899801D0899A8D
:1005300043D0630E195C07E13392339435923594BE
:10054000369E8B9A39D0640E195C03E0650E195CF7
:1005500008E18B868B8036943692369A36863698AA
:100560002BD0660E195C08E18B808B863692369410
:100570003686369A369820D0670E195C0BE1339890
:1005800035988B983696369236948B908B96369813
:10059000369A12D07A0E195C0DE1006A520E086E7E
:1005A000080E076E020E0DEC00F0339A359A496A78
:1005B000486A02D030EF05F02FEF05F0FCEF04F0B1
:1005C000600E195C26E18998899A3690338001EE95
:1005D00080F0D8901A34E926000EEA22EECF42F0DD
:1005E000EFCF43F042504F24016E43505020026E33
:1005F000000E5120036E000E5220046E04C06BF0FA
:1006000003C06AF002C069F001C068F089883590C3
:10061000F1D1610E195C26E18998899A3680338080
:1006200001EE80F0D8901A34E926000EEA22EECFCF
:1006300042F0EFCF43F042504F24016E4350502020
:10064000026E000E5120036E000E5220046E04C094
:100650006BF003C06AF002C069F001C068F0898ADB
:100660003590C8D1620E195CD8A452D036B003D0F0
:100670008998898A02D0899A89883670338001EEF8
:1006800080F0D8901A34E926000EEA22EECF42F02C
:10069000EFCF43F042504F24016E43505020026E82
:1006A000000E5120036E000E5220046E04C06BF049
:1006B00003C06AF002C069F001C068F04A5227E046
:1006C000358003EE80F0D8904A34E926000EEA2205
:1006D000EECF01F0EFCF02F00150425C02504358E0
:1006E00005E343C039F042C038F011D003EE80F08A
:1006F000D8904A34E926000EEA22EECF01F0EFCF7F
:1007000002F04250015C386E43500258396E72D18B
:10071000630E195CD8A456D0338202EE80F0D890D4
:100720001A34E926000EEA22EECF44F0EFCF45F06E
:1007300044504F24016E45505020026E000E51204F
:10074000036E000E5220046E04C06FF003C06EF002
:1007500002C06DF001C06CF0358204EE80F0D890DC
:100760001A34E926000EEA22EECF3AF0EFCF3BF042
:100770004B5221E0358403EE80F0D8904B34E926CB
:10078000000EEA22EECF3CF0EFCF3DF03C504F247C
:10079000016E3D505020026E000E5120036E000E7F
:1007A0005220046E04C073F003C072F002C071F0F6
:1007B00001C070F006D0369E359473687268716817
:1007C000706818D1640E195C2AE106EE80F01A50A8
:1007D000EB505A6E5AC000F0520E086E080E076EAB
:1007E000010E0DEC00F0010EC26E000E50EC00F098
:1007F0005B6E12C05CF0470E5C5C07E38B908B86EF
:10080000369236843696368808D0646A636A8B805E
:100810008B863692369436863698369AEBD0650EAD
:10082000195C22E106EE80F01A50EB505A6E5AC065
:1008300000F0520E086E080E076E010E0DEC00F06F
:10084000050EC26E470E5E5C07E38B968B80369476
:1008500036823696368806D08B808B8636923694D2
:1008600036863698369AC6D0660E195CD8A44DD016
:1008700006EE80F01A50EB505A6E5AC000F0520E3D
:10088000086E080E076E010E0DEC00F0368A3696E3
:1008900064521CE14E50635C19E2050EC26E010EFB
:1008A00050EC00F05D6E12C05EF0470E5E5C07E338
:1008B0008B808B96368236943696368806D08B900F
:1008C0008B8636923684369636881ED0645203E183
:1008D00063504D5C19E2010EC26E000E50EC00F048
:1008E0005B6E12C05CF0470E5C5C000107E38B8618
:1008F0008B90368436923696368806D08B968B80CF
:10090000369436823696368875D0670E195C27E1A4
:100910008B88338801EE80F0D8901A34E926000ED7
:10092000EA22EECF46F0EFCF47F046504F24016E5B
:1009300047505020026E000E5120036E000E5220D0
:10094000046E04C07BF003C07AF002C079F001C0ED
:1009500078F08B808B8636863698369A4BD07A0E16
:10096000195CD8A445D0D8901A34486E496A4936E3
:100970007F0E1A5C0AE248C000F0520E086E080EA4
:10098000076E020E0DEC00F00AD049684868006856
:10099000520E086E080E076E020E0DEC00F04C525F
:1009A00021E0358A05EE80F0D8904C34E926000E1F
:1009B000EA22EECF40F0EFCF41F040504F24016EDD
:1009C00041505020026E000E5120036E000E522046
:1009D000046E04C07FF003C07EF002C07DF001C051
:1009E0007CF005D0359A7F687E687D687C6802D08F
:1009F000196836D0196833D033D031D0A90E165CBF
:100A00000BE11B2803E114C01BF004D014C01CF040
:100A10005EEC07F025D023D0B90E165C0BE11D2843
:100A200003E114C01DF004D014C01EF0C2EC07F0A6
:100A300017D015D0C90E165C08E11F2804E114C0B8
:100A40001FF0BCEC07F00CD00AD0D90E165C07E101
:100A5000202804E114C020F0C0EC07F001D0F4D944
:100A6000060E595CD8B02BD155504F5C565050589B
:100A70005750515858505258D8A012D1588E5952E8
:100A8000D8A443D035B008D033908998899A6B6840
:100A90006A686968686838D033A01BD036B002D065
:100AA000899801D0899A38504F24016E39505020CE
:100AB000026E000E5120036E000E5220046E04C020
:100AC0006BF003C06AF002C069F001C068F03390B7
:100AD0001BD036B002D0898A01D089883670425046
:100AE0004F24016E43505020026E000E5120036EC1
:100AF000000E5220046E04C06BF003C06AF002C006
:100B000069F001C068F03380CAD0010E595C39E148
:100B100035B207D033928B9A6F686E686D686C68D7
:100B20002FD033A217D08B9A3A504F24016E3B50EE
:100B30005020026E000E5120036E000E5220046EF3
:100B400004C06FF003C06EF002C06DF001C06CF025
:100B5000339216D08B8A44504F24016E455050205A
:100B6000026E000E5120036E000E5220046E04C06F
:100B70006FF003C06EF002C06DF001C06CF0338204
:100B80008ED0020E595CD8A43ED035B406D0339432
:100B9000736872687168706835D0367E3C504F2437
:100BA000016E3D505020026E000E5120036E000E6B
:100BB0005220046E04C073F003C072F002C071F0E2
:100BC00001C070F0338436BE07D08B9A33926F68C1
:100BD0006E686D686C6816D08B8A44504F24016E25
:100BE00045505020026E000E5120036E000E522020
:100BF000046E04C06FF003C06EF002C06DF001C05F
:100C00006CF033824CD0030E595CD8B448D0040E3B
:100C1000595C09E133A806D08B9833987B687A68D1
:100C2000796878683CD0050E595C39E135BA0ED048
:100C3000339A006A520E086E080E076E020E0DEC13
:100C400000F07F687E687D687C6829D0367C36BC81
:100C500009D0006A520E086E080E076E020E0DECE7
:100C600000F009D048C000F0520E086E080E076E62
:100C7000020E0DEC00F040504F24016E4150502008
:100C8000026E000E5120036E000E5220046E04C04E
:100C90007FF003C07EF002C07DF001C07CF0D4D8AC
:100CA00052AE0CD0526A516A506A4F6A336A356A42
:100CB00000EE68F0180EEE68E82EFDD706D052AEB2
:100CC00004D0526A516A506A4F6A36A82ED080B456
:100CD0002AD0675227E1000E36B2010E136E010EC4
:100CE00036B4000E13160DE0634A642A64BE08D0C1
:100CF000645203E163507F0803E2646A7F0E636E0F
:100D00000001000E36B4010E136E010E36B2000E55
:100D1000131607E06306000E645A64AE02D0646ADC
:100D2000636A676801D0676A08D080B405D06752EB
:100D300002E16690676801D0676A36A882D00D0E1E
:100D4000C16E050EC26E010E50EC00F05D6E12C059
:100D50005EF0460EC45C16E28A8436928B9066A0E2
:100D600003D065C063F0646A36AA05D08B863684EA
:100D70003688369606D08B808B86369236943686A9
:100D8000369821D08A94000E4EBEFF0E645C07E0B8
:100D900064504E18D8B0800A800B15E003D04E5036
:100DA000635C11E3000136AA07D08B908B863684F2
:100DB00036923688369606D08B808B86369236945D
:100DC0003686369800D0010EC26E000E50EC00F050
:100DD0005B6E12C05CF0460EC45C13E28A848B9694
:100DE0003694646A636A36AA05D08B803682368868
:100DF000369606D08B808B86369236943686369819
:100E000020D08A94000E4DBEFF0E645C07E0645053
:100E10004D18D8B0800A800B04E013D063504D5CAD
:100E200010E3000136AA07D08B968B803682369469
:100E30003688369606D08B808B86368636923694E8
:100E400036988170AAEF01F05968588E156A060E1F
:100E5000155C33E2D8901534E96EEA6AEA36E93671
:100E6000EA36680EE926000EEA22EFCF01F0ECCF59
:100E700002F0ECCF03F0ECCF04F05550015C56507B
:100E80000258575003585850045815E2D89015345A
:100E9000E96EEA6AEA36E936EA36680EE926000EB5
:100EA000EA22EFCF55F0ECCF56F0ECCF57F0ECCF75
:100EB00058F015C059F0152ACAE31200620E1B5CE7
:100EC00014E11CC04AF04A520CE003EE80F0D890C6
:100ED0004A34E926000EEA22EECF38F0EFCF39F09F
:100EE00003D0396A386A359045D0630E1B5C14E133
:100EF0001CC04BF04B520CE003EE80F0D8904B340A
:100F0000E926000EEA22EECF3CF0EFCF3DF003D011
:100F10003D6A3C6A35942ED0640E1B5C06E0650E7B
:100F20001B5C03E0660E1B5C0FE106EE80F01C50BC
:100F3000EB505A6E5AC000F0520E086E080E076E43
:100F4000010E0DEC00F016D07A0E1B5C13E11CC0F4
:100F50004CF04C520CE005EE80F0D8904C34E92671
:100F6000000EEA22EECF40F0EFCF41F003D0416A0D
:100F7000406A359A1B6812001F681200216812002F
:100F8000206812001E0E1D5C35E11E520BE1356A11
:100F9000396A386A4A6A4B6A3D6A3C6A416A406A01
:100FA0004C6A27D01EC04AF003EE80F0D8901E3461
:100FB000E926000EEA22EECF38F0EFCF39F01EC05E
:100FC0004BF003EE80F0D8901E34E926000EEA22A2
:100FD000EECF3CF0EFCF3DF01EC04CF005EE80F0C0
:100FE000D8901E34E926000EEA22EECF40F0EFCF73
:100FF00041F092D0420E1D5C07E11E5203E1349095
:101000008DD801D0348088D0460E1D5C09E1336A4A
:10101000356A8998899A8B988B9A8B92ADD87CD0B7
:10102000470E1D5C07E18B968B9036943692369670
:10103000369872D0480E1D5C15E106EE80F01E5009
:10104000EB505A6E5AC000F0520E086E080E076E32
:10105000010E0DEC00F08B808B963682369436961E
:1010600036885AD0490E1D5C15E106EE80F01E5000
:10107000EB505A6E5AC000F0520E086E080E076E02
:10108000010E0DEC00F08B908B86369236843696EE
:10109000368842D04A0E1D5C0FE11EC04DF066A09E
:1010A00005D04E50655C02E265C04EF04E504D5C7E
:1010B00002E34D284E6E30D04B0E1D5C0FE11EC07A
:1010C0004EF066A005D04E50655C02E265C04EF061
:1010D0004E504D5C02E34D284E6E1ED07B0E1D5CC3
:1010E0001BE1336A356A8998899A8B988B9A949018
:1010F0008B9094968B96366A0068520E086E080E96
:10110000076E010E0DEC00F0006A520E086E080E1C
:10111000076E020E0DEC00F01D681200336A356A8E
:101120008998899A8B988B9A94908B9094968B96A9
:101130000068520E086E080E076E010E0DEC00F0EE
:10114000006A520E086E080E076E020E0DEC00F0DB
:101150005A684D6A66A003D065C04EF002D07F0E7B
:101160004E6E366A4A6A4B6A4C6A396A386A3D6A18
:101170003C6A416A406A12000068520E086E080E0E
:10118000076E010E0DEC00F0010EC26E000E50EC69
:1011900000F05B6E12C05CF0460EC45C0AE28B800D
:1011A0008B86646A636A4D6A3692369436863698C0
:1011B0001200050EC26E010E50EC00F05D6E12C002
:1011C0005EF0460EC45C10E28B908B8636923684BD
:1011D0003696368866A004D065C063F0646A03D092
:1011E000646A7F0E636E06D08B908B86369236844F
:1011F00036963688FC0E006E520E086E080E076E8C
:10120000010E0DEC00F0030EC26E000E50EC00F06B
:101210005B6E12C05CF0470EC45C09E3010EC26E47
:10122000000E50EC00F05B6E12C05CF0F4D78B80C7
:101230003692369436863698646A636A369A66A021
:1012400001D8120064506310D8A496DFFC0E006E23
:10125000520E086E080E076E010E0DEC00F08B802A
:101260008B963694368236963688050EC26E010EFF
:1012700050EC00F05D6E12C05EF0470EC45C12E3ED
:10128000050EC26E010E50EC00F05D6E12C05EF0F5
:1012900080B406D0675203E1634A642A676801D0CC
:1012A000676AEBD763C065F0668066D70301816922
:1012B00080695C0E836F7A0E826F590E856F850E82
:1012C000846F580E876F140E866F560E896FA90EA5
:1012D000886F550E8B6F430E8A6F530E8D6FE30E22
:1012E0008C6F520E8F6F890E8E6F510E916F350E6F
:1012F000906F4F0E936FE60E926F4E0E956F9C0E91
:10130000946F4D0E976F580E966F4C0E996F190E85
:10131000986F4A0E9B6FDF0E9A6F490E9D6FAA0E53
:101320009C6F480E9F6F7A0E9E6F470EA16F4F0EF7
:10133000A06F460EA36F290EA26F450EA56F080E73
:10134000A46F430EA76FEB0EA66F420EA96FD30ECC
:10135000A86F410EAB6FBF0EAA6F400EAD6FB00EFF
:10136000AC6F3F0EAF6FA50EAE6F3E0EB16F9E0E0F
:10137000B06F3D0EB36F9C0EB26F3C0EB56F9E0EFC
:10138000B46F3B0EB76FA40EB66F3A0EB96FAE0EC8
:10139000B86F390EBB6FBC0EBA6F380EBD6FCE0E74
:1013A000BC6F370EBF6FE30EBE6F360EC16FFD0E02
:1013B000C06F360EC36F1A0EC26F350EC56F3B0E6F
:1013C000C46F340EC76F5F0EC66F330EC96F870EC2
:1013D000C86F320ECB6FB20ECA6F310ECD6FE10EF9
:1013E000CC6F310ECF6F140ECE6F300ED16F490E11
:1013F000D06F2F0ED36F820ED26F2E0ED56FBE0E12
:10140000D46F2D0ED76FFD0ED66F2D0ED96F3F0EF8
:10141000D86F2C0EDB6F850EDA6F2B0EDD6FCD0EC5
:10142000DC6F2B0EDF6F180EDE6F2A0EE16F670E7A
:10143000E06F290EE36FB80EE26F290EE56F0C0E18
:10144000E46F280EE76F620EE66F270EE96FBC0EA1
:10145000E86F270EEB6F180EEA6F260EED6F760E13
:10146000EC6F250EEF6FD80EEE6F250EF16F3C0E70
:10147000F06F240EF36FA20EF26F240EF56F0B0EB9
:10148000F46F230EF76F760EF66F220EF96FE40EEF
:10149000F86F220EFB6F540EFA6F210EFD6FC60E11
:1014A000FC6F210EFF6F3B0EFE6F200E0401016FDB
:1014B000B20E006F200E036F2B0E026F1F0E056F12
:1014C000A60E046F1F0E076F240E066F1E0E096F07
:1014D000A30E086F1E0E0B6F250E0A6F1D0E0D6FEB
:1014E000A90E0C6F1D0E0F6F2E0E0E6F1C0E116FBE
:1014F000B60E106F1C0E136F3F0E126F1B0E156F82
:10150000CB0E146F1B0E176F580E166F1A0E196F35
:10151000E80E186F1A0E1B6F790E1A6F1A0E1D6FD8
:101520000B0E1C6F190E1F6FA00E1E6F190E216F70
:10153000360E206F180E236FCE0E226F180E256FF9
:10154000680E246F180E276F030E266F170E296F73
:10155000A00E286F170E2B6F3F0E2A6F160E2D6FE1
:10156000DF0E2C6F160E2F6F800E2E6F160E316F42
:10157000240E306F150E336FC80E326F150E356F97
:101580006E0E346F150E376F160E366F140E396FE0
:10159000BF0E386F140E3B6F690E3A6F140E3D6F1D
:1015A000150E3C6F130E3F6FC20E3E6F130E416F50
:1015B000710E406F130E436F210E426F120E456F76
:1015C000D20E446F120E476F840E466F120E496F93
:1015D000380E486F110E4B6FED0E4A6F110E4D6FA6
:1015E000A30E4C6F110E4F6F5A0E4E6F110E516FAE
:1015F000120E506F100E536FCC0E526F100E556FAF
:10160000870E546F100E576F420E566F0F0E596FA4
:1016100058695B6FBD0E5A6F0F0E5D6F7C0E5C6F6D
:101620000F0E5F6F3D0E5E6F0E0E616FFE0E606FF0
:101630000E0E636FC00E626F0E0E656F830E646FC9
:101640000E0E676F470E666F0E0E696F0C0E686F99
:101650000D0E6B6FD20E6A6F0D0E6D6F990E6C6F63
:101660000D0E6F6F610E6E6F0D0E716F2A0E706F23
:101670000C0E736FF40E726F0C0E756FBE0E746FDE
:101680000C0E776F8A0E766F0C0E796F560E786F90
:101690000C0E7B6F230E7A6F0B0E7D6FF10E7C6F3D
:1016A0000B0E7F6FC00E7E6F050181698069A20EEF
:1016B000836FC30E826F9A0E856F460E846F960EEF
:1016C000876F320E866F920E896F3A0E886F8E0E7C
:1016D0008B6F5D0E8A6F8A0E8D6F9A0E8C6F860EE1
:1016E0008F6FF00E8E6F830E916F5F0E906F7F0E77
:1016F000936FE70E926F7C0E956F850E946F790E47
:10170000976F3B0E966F760E996F070E986F720E5D
:101710009B6FE80E9A6F6F0E9D6FDF0E9C6F6C0EC5
:101720009F6FEA0E9E6F6A0EA16F0A0EA06F670E82
:10173000A36F3C0EA26F640EA56F820EA46F610EA4
:10174000A76FDA0EA66F5F0EA96F440EA86F5C0E2E
:10175000AB6FBF0EAA6F5A0EAD6F4C0EAC6F570E2B
:10176000AF6FE90EAE6F550EB16F960EB06F530EA0
:10177000B36FB26F510EB56F200EB46F4E0EB76FD0
:10178000FB0EB66F4C0EB96FE50EB86F4A0EBB6F0D
:10179000DC0EBA6F480EBD6FE20EBC6F460EBF6F17
:1017A000F50EBE6F450EC16F150EC06F430EC36FB1
:1017B000420EC26F410EC56F7B0EC46F3F0EC76FE6
:1017C000C00EC66F3E0EC96F100EC86F3C0ECB6FB9
:1017D0006D0ECA6F3A0ECD6FD40ECC6F390ECF6F2F
:1017E000460ECE6F370ED16FC20ED06F360ED36F4E
:1017F000490ED26F340ED56FDA0ED46F330ED76F19
:10180000740ED66F320ED96F180ED86F300EDB6F94
:10181000C50EDA6F2F0EDD6F7B0EDC6F2E0EDF6FC5
:101820003A0EDE6F2D0EE16F020EE06F2B0EE36FAE
:10183000D10EE26F2A0EE56FA90EE46F290EE76F55
:10184000880EE66F280EE96F6F0EE86F270EEB6FBC
:101850005E0EEA6F260EED6F530EEC6F250EEF6FE6
:10186000500EEE6F240EF16F540EF06F230EF36FD7
:101870005E0EF26F220EF56F6F0EF46F210EF76F92
:10188000860EF66F200EF96FA30EF86F1F0EFB6F1A
:10189000C60EFA6F1E0EFD6FEF0EFC6F1E0EFF6F71
:1018A000FE6F1D0E0601016F520E006F1C0E036FBE
:1018B0008C0E026F1B0E056FCB0E046F1B0E076F95
:1018C0000F0E066F1A0E096F580E086F190E0B6F68
:1018D000A50E0A6F180E0D6FF80E0C6F180E0F6F15
:1018E0004F0E0E6F170E116FAB0E106F170E136F9A
:1018F0000A0E126F160E156F6F0E146F150E176FFE
:10190000D70E166F150E196F430E186F140E1B6F3E
:10191000B30E1A6F140E1D6F270E1C6F130E1F6F60
:101920009F0E1E6F130E216F1A0E206F120E236F63
:10193000990E226F120E256F1B0E246F110E276F4A
:10194000A10E266F110E296F290E286F100E2B6F16
:10195000B50E2A6F100E2D6F440E2C6F0F0E2F6FC9
:10196000D60E2E6F0F0E316F6B0E306F0F0E336F62
:10197000030E326F0E0E356F9D0E346F0E0E376FE5
:101980003A0E366F0D0E396FDA0E386F0D0E3B6F53
:101990007C0E3A6F0D0E3D6F210E3C6F0C0E3F6FAB
:1019A000C80E3E6F0C0E416F720E406F0C0E436FEF
:1019B0001E0E426F0B0E456FCC0E446F0B0E476F21
:1019C0007C0E466F0B0E496F2E0E486F0A0E4B6F42
:1019D000E30E4A6F0A0E4D6F990E4C6F0A0E4F6F51
:1019E000510E4E6F0A0E516F0B0E506F090E536F52
:1019F000C80E526F090E556F850E546F090E576F42
:101A0000450E566F090E596F060E586F080E5B6F24
:101A1000C90E5A6F080E5D6F8E0E5C6F080E5F6FF9
:101A2000540E5E6F080E616F1C0E606F070E636FC1
:101A3000E50E626F070E656FAF0E646F070E676F7E
:101A40007B0E666F070E696F490E686F070E6B6F2E
:101A5000170E6A6F060E6D6FE70E6C6F060E6F6FD6
:101A6000B90E6E6F060E716F8B0E706F060E736F70
:101A70005F0E726F060E756F340E746F060E776F01
:101A80000A0E766F050E796FE10E786F050E7B6F8B
:101A9000B90E7A6F050E7D6F930E7C6F050E7F6F0A
:101AA0006D0E7E6F00011200040E0101836F880E1F
:101AB000826F040E856FA60E846F040E876FB60EBC
:101AC000866F040E896FC60E886F040E8B6FD60E5C
:101AD0008A6F040E8D6FE60E8C6F040E8F6FF60EFC
:101AE0008E6F050E916F070E906F050E936F170E98
:101AF000926F050E956F280E946F050E976F390E35
:101B0000966F050E996F4B0E986F050E9B6F5D0ECD
:101B10009A6F050E9D6F6E0E9C6F050E9F6F800E67
:101B20009E6F050EA16F930EA06F050EA36FA50EFD
:101B3000A26F050EA56FB80EA46F050EA76FCB0E92
:101B4000A66F050EA96FDF0EA86F050EAB6FF20E24
:101B5000AA6F060EAD6FAC6FAF6F1A0EAE6F060EAA
:101B6000B16F2E0EB06F060EB36F430EB26F060E3E
:101B7000B56F580EB46F060EB76F6D0EB66F060ECA
:101B8000B96F830EB86F060EBB6F980EBA6F060E54
:101B9000BD6FAE0EBC6F060EBF6FC40EBE6F060EDD
:101BA000C16FDB0EC06F060EC36FF20EC26F070E61
:101BB000C56F090EC46F070EC76F210EC66F070EE3
:101BC000C96F380EC86F070ECB6F500ECA6F070E65
:101BD000CD6F690ECC6F070ECF6F810ECE6F070EE3
:101BE000D16F9A0ED06F070ED36FB40ED26F070E5F
:101BF000D56FCD0ED46F070ED76FE70ED66F080ED8
:101C0000D96F020ED86F080EDB6F1D0EDA6F080E4B
:101C1000DD6F380EDC6F080EDF6F530EDE6F080EBF
:101C2000E16F6F0EE06F080EE36F8B0EE26F080E30
:101C3000E56FA70EE46F080EE76FC40EE66F080E9F
:101C4000E96FE10EE86F080EEB6FEA69090EED6FC0
:101C50001D0EEC6F090EEF6F3B0EEE6F090EF16F6C
:101C60005A0EF06F090EF36F790EF26F090EF56FD1
:101C7000990EF46F090EF76FB90EF66F090EF96F32
:101C8000D90EF86F090EFB6FFA0EFA6F0A0EFD6F90
:101C90001B0EFC6F0A0EFF6F3D0EFE6F0A0E020157
:101CA000016F5F0E006F0A0E036F820E026F0A0E45
:101CB000056FA50E046F0A0E076FC80E066F0A0E99
:101CC000096FEC0E086F0B0E0B6F110E0A6F0B0EE7
:101CD0000D6F360E0C6F0B0E0F6F5B0E0E6F0B0E33
:101CE000116F810E106F0B0E136FA70E126F0B0E7C
:101CF000156FCE0E146F0B0E176FF50E166F0C0EC0
:101D0000196F1D0E186F0C0E1B6F460E1A6F0C0EFE
:101D10001D6F6F0E1C6F0C0E1F6F980E1E6F0C0E3A
:101D2000216FC20E206F0C0E236FED0E226F0D0E71
:101D3000256F180E246F0D0E276F430E266F0D0EA4
:101D4000296F700E286F0D0E2B6F9C0E2A6F0D0ED3
:101D50002D6FCA0E2C6F0D0E2F6FF80E2E6F0E0EFC
:101D6000316F260E306F0E0E336F550E326F0E0E22
:101D7000356F850E346F0E0E376FB60E366F0E0E42
:101D8000396FE70E386F0F0E3B6F180E3A6F0F0E5C
:101D90003D6F4B0E3C6F0F0E3F6F7E0E3E6F0F0E72
:101DA000416FB10E406F0F0E436FE60E426F100E83
:101DB000456F1B0E446F100E476F500E466F100E8E
:101DC000496F870E486F100E4B6FBE0E4A6F100E94
:101DD0004D6FF60E4C6F110E4F6F2E0E4E6F110E93
:101DE000516F680E506F110E536FA20E526F110E8D
:101DF000556FDC0E546F120E576F180E566F120E81
:101E0000596F540E586F120E5B6F910E5A6F120E6F
:101E10005D6FCF0E5C6F130E5F6F0E0E5E6F130E55
:101E2000616F4D0E606F130E636F8E0E626F130E37
:101E3000656FCF0E646F140E676F110E666F140E10
:101E4000696F540E686F140E6B6F980E6A6F140EE4
:101E50006D6FDC0E6C6F150E6F6F220E6E6F150EB0
:101E6000716F680E706F150E736FB00E726F150E76
:101E7000756FF80E746F160E776F410E766F160E33
:101E8000796F8C0E786F160E7B6FD70E7A6F170EE8
:101E90007D6F230E7C6F170E7F6F700E7E6F0001BB
:101EA0001200160E0401836F500E826F160E856F9E
:101EB000230E846F150E876FF60E866F150E896FD1
:101EC000C90E886F150E8B6F9C0E8A6F150E8D6F65
:101ED0006F0E8C6F150E8F6F420E8E6F150E916FF9
:101EE000906F140E936FE80E926F140E956FBB0EE9
:101EF000946F140E976F8E0E966F140E996F610E7D
:101F0000986F140E9B6F340E9A6F140E9D6F070E10
:101F10009C6F130E9F6FDA0E9E6F130EA16FAD0EA6
:101F2000A06F130EA36F800EA26F130EA56F530E3A
:101F3000A46F130EA76F260EA66F120EA96FF90ECF
:101F4000A86F120EAB6FCC0EAA6F120EAD6F9F0E64
:101F5000AC6F120EAF6F720EAE6F120EB16F450EF8
:101F6000B06F120EB36F180EB26F110EB56FEB0E8D
:101F7000B46F110EB76FBE0EB66F110EB96F910E22
:101F8000B86F110EBB6F640EBA6F110EBD6F370EB6
:101F9000BC6F110EBF6F0A0EBE6F100EC16FDD0E4B
:101FA000C06F100EC36FB00EC26F100EC56F830EE0
:101FB000C46F100EC76F560EC66F100EC96F290E74
:101FC000C86F0F0ECB6FFC0ECA6F0F0ECD6FCF0E0A
:101FD000CC6F0F0ECF6FA20ECE6F0F0ED16F750E9E
:101FE000D06F0F0ED36F480ED26F0F0ED56F1B0E32
:101FF000D46F0E0ED76FEE0ED66F0E0ED96FC10EC8
:10200000D86F0E0EDB6F940EDA6F0E0EDD6F670E5B
:10201000DC6F0E0EDF6F3A0EDE6F0E0EE16F0D0EEF
:10202000E06FE36FE00EE26F0D0EE56FB30EE46F4D
:102030000D0EE76F860EE66F0D0EE96F590EE86F15
:102040000D0EEB6F2C0EEA6F0C0EED6FEC69EF6F5F
:10205000D20EEE6F0C0EF16FA50EF06F0C0EF36F3B
:10206000780EF26F0C0EF56F4B0EF46F0C0EF76FCF
:102070001E0EF66F0B0EF96FF10EF86F0B0EFB6F65
:10208000C40EFA6F0B0EFD6F970EFC6F0B0EFF6FF9
:102090006A0EFE6F0B0E0501016F3D0E006F0B0EF9
:1020A000036F100E026F0A0E056FE30E046F0A0E27
:1020B000076FB60E066F0A0E096F890E086F0A0EBB
:1020C0000B6F5C0E0A6F0A0E0D6F2F0E0C6F0A0E4F
:1020D0000F6F020E0E6F090E116FD50E106F090EE5
:1020E000136FA80E126F090E156F7B0E146F090E79
:1020F000176F4E0E166F090E196F210E186F080E0E
:102100001B6FF40E1A6F080E1D6FC70E1C6F080EA2
:102110001F6F9A0E1E6F080E216F6D0E206F080E36
:10212000236F400E226F080E256F130E246F070ECB
:10213000276FE60E266F070E296FB90E286F070E60
:102140002B6F8C0E2A6F070E2D6F5F0E2C6F070EF4
:102150002F6F320E2E6F070E316F050E306F060E89
:10216000336FD80E326F060E356FAB0E346F060E1E
:10217000376F7E0E366F060E396F510E386F060EB2
:102180003B6F240E3A6F050E3D6FF70E3C6F050E48
:102190003F6FCA0E3E6F050E416F9D0E406F050EDC
:1021A000436F700E426F050E456F430E446F050E70
:1021B000476F160E466F040E496FE90E486F040E06
:1021C0004B6FBC0E4A6F040E4D6F8F0E4C6F040E9A
:1021D0004F6F620E4E6F040E516F350E506F040E2E
:1021E000536F080E526F030E556FDB0E546F030EC4
:1021F000576FAE0E566F030E596F810E586F030E58
:102200005B6F540E5A6F030E5D6F270E5C6F020EEC
:102210005F6FFA0E5E6F020E616FCD0E606F020E81
:10222000636FA00E626F020E656F730E646F020E15
:10223000676F460E666F020E696F190E686F010EAA
:102240006B6FEC0E6A6F010E6D6FBF0E6C6F010E3F
:102250006F6F920E6E6F010E716F650E706F010ED3
:10226000736F380E726F010E756F0B0E746F776B94
:10227000DE0E766F796BB10E786F7B6B840E7A6FA2
:102280007D6B570E7C6F7F6B2A0E7E6F050E0201F1
:10229000836F940E826F050E856FC10E846F050EDD
:1022A000876FEE0E866F060E896F1B0E886F060E07
:1022B0008B6F480E8A6F060E8D6F750E8C6F060E33
:1022C0008F6FA20E8E6F060E916FCF0E906F060E5F
:1022D000936FFC0E926F070E956F290E946F070E89
:1022E000976F560E966F070E996F830E986F070EB5
:1022F0009B6FB00E9A6F070E9D6FDD0E9C6F080EE0
:102300009F6F0A0E9E6F080EA16F370EA06F080E0A
:10231000A36F640EA26F080EA56F910EA46F080E36
:10232000A76FBE0EA66F080EA96FEB0EA86F090E61
:10233000AB6F180EAA6F090EAD6F450EAC6F090E8C
:10234000AF6F720EAE6F090EB16F9F0EB06F090EB8
:10235000B36FCC0EB26F090EB56FF90EB46F0A0EE3
:10236000B76F260EB66F0A0EB96F530EB86F0A0E0E
:10237000BB6F800EBA6F0A0EBD6FAD0EBC6F0A0E3A
:10238000BF6FDA0EBE6F0B0EC16F070EC06F0B0E64
:10239000C36F340EC26F0B0EC56F610EC46F0B0E90
:1023A000C76F8E0EC66F0B0EC96FBB0EC86F0B0EBC
:1023B000CB6FE80ECA6F0C0ECD6F150ECC6F0C0EE6
:1023C000CF6F420ECE6F0C0ED16F6F0ED06F0C0E12
:1023D000D36F9C0ED26F0C0ED56FC90ED46F0C0E3E
:1023E000D76FF60ED66F0D0ED96F230ED86F0D0E68
:1023F000DB6F500EDA6F0D0EDD6F7D0EDC6F0D0E94
:10240000DF6FAA0EDE6F0D0EE16FD70EE06F0E0EBE
:10241000E36F040EE26F0E0EE56F310EE46F0E0EE9
:10242000E76F5E0EE66F0E0EE96F8B0EE86F0E0E15
:10243000EB6FB80EEA6F0E0EED6FE50EEC6F0F0E40
:10244000EF6F120EEE6F0F0EF16F3F0EF06F0F0E6B
:10245000F36F6C0EF26F0F0EF56F990EF46F0F0E97
:10246000F76FC60EF66F0F0EF96FF30EF86F100EC2
:10247000FB6F200EFA6F100EFD6F4D0EFC6F100EED
:10248000FF6F7A0EFE6F100E0301016FA70E006F33
:10249000100E036FD40E026F110E056F010E046F44
:1024A000110E076F2E0E066F110E096F5B0E086F6F
:1024B000110E0B6F880E0A6F110E0D6FB50E0C6F9B
:1024C000110E0F6FE20E0E6F120E116F0F0E106FC6
:1024D000120E136F3C0E126F120E156F690E146FF1
:1024E000120E176F960E166F120E196FC30E186F1D
:1024F000120E1B6FF00E1A6F130E1D6F1D0E1C6F48
:10250000130E1F6F4A0E1E6F130E216F770E206F72
:10251000130E236FA40E226F130E256FD10E246F9E
:10252000130E276FFE0E266F140E296F2B0E286FC9
:10253000140E2B6F580E2A6F140E2D6F850E2C6FF4
:10254000140E2F6FB20E2E6F140E316FDF0E306F20
:10255000150E336F0C0E326F150E356F390E346F4A
:10256000150E376F660E366F150E396F930E386F76
:10257000150E3B6FC00E3A6F150E3D6FED0E3C6FA2
:10258000160E3F6F1A0E3E6F160E416F470E406FCC
:10259000160E436F740E426F160E456FA10E446FF8
:1025A000160E476FCE0E466F160E496FFB0E486F24
:1025B000170E4B6F280E4A6F170E4D6F550E4C6F4E
:1025C000170E4F6F820E4E6F170E516FAF0E506F7A
:1025D000170E536FDC0E526F180E556F090E546FA5
:1025E000180E576F360E566F180E596F630E586FD0
:1025F000180E5B6F900E5A6F180E5D6FBD0E5C6FFC
:10260000180E5F6FEA0E5E6F190E616F170E606F26
:10261000190E636F440E626F190E656F710E646F51
:10262000190E676F9E0E666F190E696FCB0E686F7D
:10263000190E6B6FF80E6A6F1A0E6D6F250E6C6FA8
:102640001A0E6F6F520E6E6F1A0E716F7F0E706FD3
:102650001A0E736FAC0E726F1A0E756FD90E746FFF
:102660001B0E776F060E766F1B0E796F330E786F29
:102670001B0E7B6F600E7A6F1B0E7D6F8D0E7C6F55
:102680001B0E7F6FBA0E7E6F00011200060180697B
:10269000FE0E816F826FFD0E836F846F856FFC0E5F
:1026A000866F876F886FFB0E896F8A6F8B6F8C6F59
:1026B000FA0E8D6F8E6F8F6FF90E906F916F926F14
:1026C000F80E936F946F956FF70E966F976F986FE4
:1026D000F60E996F9A6F9B6FF50E9C6F9D6FF40EBF
:1026E0009E6F9F6FF30EA06FA16FF20EA26FA36F8C
:1026F000F10EA46FA56FF00EA66FA76FEF0EA86F77
:10270000A96FEE0EAA6FAB6FED0EAC6FAD6FEC0E56
:10271000AE6FAF6FEB0EB06FB16FEA0EB26FB36F0B
:10272000E90EB46FB56FE80EB66FB76FE70EB86F0E
:10273000B96FE60EBA6FBB6FE50EBC6FBD6FE40EEE
:10274000BE6FBF6FE30EC06FC16FE20EC26FC36F8B
:10275000E10EC46FC56FE00EC66FC76FDF0EC86FA6
:10276000C96FDE0ECA6FCB6FDD0ECC6FCD6FDC0E86
:10277000CE6FCF6FDB0ED06FD16FDA0ED26FD36F0B
:10278000D90ED46FD56FD80ED66FD76FD70ED86F3E
:10279000D96FD60EDA6FDB6FD50EDC6FDD6FD40E1E
:1027A000DE6FDF6FD30EE06FE16FD20EE26FE36F8B
:1027B000D10EE46FE56FD00EE66FE76FCF0EE86FD6
:1027C000E96FCE0EEA6FEB6FCD0EEC6FED6FCC0EB6
:1027D000EE6FEF6FCB0EF06FF16FCA0EF26FF36F0B
:1027E000C90EF46FF56FC80EF66FF76FC70EF86F6E
:1027F000F96FC60EFA6FFB6FC50EFC6FFD6FC40E4E
:0A280000FE6FFF6F00011200FFD70A
:020000040030CA
:0300010006160ED2
:020005008580F4
:060008000FC00FE00F40E5
:00000001FF
